:030000000210A14A
:03000B000200A24E
:03002B000202CB03
:03005B0002041587
:030073000203EF96
:1000800002030406080C10182030406080040608A3
:100090000C10182030406080A0C005050D0502033B
:1000A0000302C2AFC0D0C0E020622C20680241B77A
:1000B0003066024177302F02E4730563C3740595FF
:1000C0002540F5956340F12069EE758A78E5257045
:1000D00003758A000202C485258AC262E525F47090
:1000E00002213E206802212B758B00D0E0D0D0D2B7
:1000F00097D295D293D2AF32D297D295D29374063B
:10010000D5E0FDE53C1420E21520E10D207D02D272
:1001100092307D02D29602013BD29402013B207DB7
:1001200002D296307D02D29202013B758B00D0E064
:10013000D0D0D297D295D293D2AF32758B00D0E087
:10014000D0D0D2AF3241B7E525600A207D02C297F8
:10015000307D02C293D29541B7E5256002C2952059
:100160007D02D293307D02D29741B7E525600A2007
:100170007D02C293307D02C297207D02D297307DEE
:1001800002D29341B7207D02C296307D02C29220F6
:100190007D02C292307D02C2967406D5E0FDE5254F
:1001A000600A207D02C297307D02C293D29541B78A
:1001B000207D02C296307D02C292C2947406D5E0C0
:1001C000FDE525600A207D02C297307D02C293D2F0
:1001D0009541B7C294207D02C296307D02C29274CE
:1001E00006D5E0FDE5256002C295207D02D2933060
:1001F0007D02D29741B7C294207D02C292307D0227
:10020000C2967406D5E0FDE5256002C295207D0208
:10021000D293307D02D29741B7207D02C292307DC9
:1002200002C296C2947406D5E0FDE525600A207DE1
:1002300002C293307D02C297207D02D297307D02A8
:10024000D29341B7207D02C292307D02C296207DBA
:1002500002C296307D02C2927406D5E0FDE52560AB
:100260000A207D02C293307D02C297207D02D29780
:10027000307D02D29341B730723DE53C20E21A2036
:10028000E129207D02C296307D02C292207D02C209
:1002900092307D02C2960202B720E1E6207D02C2C2
:1002A00096307D02C292C2940202B7C294207D02AF
:1002B000C292307D02C296E525F4F58A758B0075F1
:1002C0006300D262D0E0D0D0D2AF32C2AFC2AD5361
:1002D000E6EFC0D0C0E0D2D3D2AFC2CEE5296007EE
:1002E0002074461529612978007900E580307E0167
:1002F000F430E50278FF53DACF207E0343DA203072
:100300007E0343DA10C2D8C271E580307E01F4303A
:10031000E50279FFC3E89970CE3061037529182092
:1003200074037529188859D270E52A6004152A616A
:100330003920740543DA01C2D82070026194A859AB
:10034000206102C270207431C3E894F0400374F05D
:10035000F8E8C4540F28F87984B703026179C3130D
:10036000C3138721200802C313200A06C3C898F8C4
:10037000617928F8500374FFF8C3E895625003E5EB
:1003800062F8882230690AC3E522955E4003855EE3
:1003900022852224A824C3E524955E4002A85E8815
:1003A00025C3E52594404002D26420CF0CD0E0D094
:1003B000D0C2D343E610D2AD32C2CF7801E5296076
:1003C000053074021529C3E55994014005755C0098
:1003D00061E3755D00756400E55C2401F55C500324
:1003E000755CFFD0E0D0D0C2D343E610D2AD32C0AE
:1003F000D0C0E0C2AF53917F53E67FC260759100D9
:10040000C3E49550F594E49551F595759104D0E0C9
:10041000D0D0D2AF32C2AF53E6EFC2ADC0D0C0E051
:10042000C0F0D2D3D2AFA8FBA9FCC2D830710281F0
:100430007C53DACF207E0343DA10307E0343DA2088
:10044000D271E580307E01F420E50281538826894F
:1004500027C1B853DACF207E0343DA20307E03432E
:10046000DA10C2D8C271307402C1A47800E58030BD
:0F0470007E01F430E502C1A48859C18B53DACF65
:10047F00207E0343DA20307E0343DA10C2712061FD
:10048F0002A14C53DACF207E0343DA10307E0343B0
:10049F00DA20C2D8D27188548955C3E89552F8E949
:1004AF009553F9E4FB7E027A00C3E8948CE994003B
:1004BF005005755800A13CC3E894C8E99400500852
:1004CF00E4D2E4FB7A0AA119C3E89468E9940150D5
:1004DF0008E4D2E3FB7A0FA119C3E894D0E99402A0
:1004EF005008E4D2E2FB7A1EA119C3E894A0E99464
:1004FF00055008E4D2E1FB7A3CA119C3E89498E9CE
:10050F0094085008E4D2E0FB7A787E00C3E8955651
:10051F00FCE99557FD30E708ECF42401FCEDF4FD00
:10052F00755800C3EC9AED9E500375580188568993
:10053F0057A854A955885289537802C18BC3E8959F
:10054F0026F8E99527F9307C02C16F307B02C16F25
:10055F00307A02C168207502A16FE9FDE8FCA18E17
:10056F00E9C313F9E813F8307902C168E9C313F945
:10057F00E813F8307802C168E9C313FDE813FC20D3
:10058F006126C3EC941CED94024002A1A5ED7018F6
:10059F00C3EC94C850120528C3E528940A5002C131
:1005AF00A4755900D270C1A4E52860021528740003
:1005BF00207F0B7888E67896B40302789EE624FABB
:1005CF00FEE43400FFC3EC9EFCED9FFD920878889B
:1005DF00E6B40327A2085009207D20C2AFD27DA127
:1005EF00F7307D17C2AFC27DD297D295D293C29604
:1005FF00C294C292206902D26BD2AFA2085017E602
:10060F00B4030DECF42401FCEDF43400FD020625D7
:10061F0078007900C16F7888E6B40315EC33FCEDF0
:10062F0033FDC3EC940AFCED9400FD50047C007D77
:10063F0000C3EC94FFED9400400678FF7900C16F82
:10064F00EC856FF0A4C5F0A2F733F87900400302F0
:10065F00068B78FF790002068BE9C313F9E813F8CC
:10066F00307C0EE9600278FFC3E81338F8E43400F9
:10067F00F9C3E894FFE99400400278FF8859D270DB
:10068F00206102C1A4741FF4552F4BF52FC274E4DF
:10069F002B7002D27475291830740375290A3061D2
:1006AF0002C1B820740353DAFE752A06307403753D
:1006BF002A0AD0F0D0E0D0D0C2D3D2AD43E6103268
:1006CF0079010206ED79030206ED790A0206ED794A
:1006DF001E0206ED79640206ED79C80206ED781761
:1006EF00E4D5E0FDD8FAD9F6227A147B7802071404
:1006FF007A107B8C0207147A0D7BB40207147A0BE5
:10070F007BC8020714AC257525017902B27DE4C2BE
:10071F0094D5E0FDE5256002C295D5E0FDD295D5D3
:10072F00E0FDD294D5E0FDE525600A207D02C29759
:10073F00307D02C293E570D5E0FD207D02D2973067
:10074F007D02D2937496D5E0FDD9C1EAF8D5E0FDCC
:10075F00D8FBDBB1C2948C2522C37C007D0075F0E1
:10076F000005F0EA33FAEB33FB50F6EB13FBEA1319
:10077F00FAC3E9FFE8FEE89AF8E99BF95004EFF9AC
:10078F00EEF8B3EC33FCED33FDD5F0DFEDF9ECF81B
:10079F0022E889F08A20D2D4F8A9F07B0030F70B39
:1007AF007BFFF42401F8E9F43400F9E88520F0A484
:1007BF00ADF0F8E98520F0A4AFF0FEED2EF974004E
:1007CF003FFA7C04C3EA13FAE913F9E813F8DCF4EF
:1007DF008BF030F70AE8F42401F8E9F43400F9E873
:1007EF0089F0C2D4F8A9F02222E547603BC3E53B6C
:1007FF0013F9E53A13F8C3E53E98F8E53F99F95038
:10080F000CC3E89480E994FF4016020833C3E894C0
:10081F007FE994005003020833787F790002083390
:10082F00788079FF8843894422E5476058E543255E
:10083F0040F8E5443541F9854420E4300701F435AB
:10084F0042FA30E709C3EA94F04015020875C3EA8B
:10085F00940F500302087578FF79FF7A0F0208751D
:0F086F00780079007AF0C3E524955E5006E52401
:10087E006009018EE54420E70D018EE54430E70660
:10088E00884089418A4222E54770030208F978A11F
:10089E00E6FAC3E54333F8E54433F91207A0E9302D
:1008AE00E70BC3E89480E994FF401301D0C3E894AA
:1008BE007FE99400500201D0787F790001D07880D2
:1008CE0079FFE820E715C3E52398F84009C3E894BB
:1008DE000140030208F778010208F7E8F424012525
:1008EE0023F840030208F778FF884522E547700396
:1008FE0002095C78A2E6FAA841A9421207A0E930E3
:10090E00E70CC3E89401E994FF4016020933C3E8EB
:10091E0094FFE99400500302093378FF790002092D
:10092E0033780179FFE920E715C3E54598F84009CA
:10093E00C3E89401400302095A780002095AE8F408
:10094E0024012545F8400302095A78FF88242278AD
:10095E00FFC264E52D5406702FD264C3E53B940AA2
:10096E004009C3E52594405002C264E53B6019740A
:10097E00FF853BF0848537F0A4F8C5F0600278FF60
:10098E00C3E895615002A861886022020A36788316
:10099E00E6F520120EAF75E8901206CF75E890E5D9
:1009AE00E820ECFBA8BDA9BE120F5D756B55756CEA
:1009BE0000C3740013FD745513FC74552CFC7400A5
:1009CE003DFDECFAEDFBC3E89AE99B4014E56B2480
:1009DE0055F56BE56C3400F56CEA2CFAEB3DFB80BB
:1009EE00E5AE6BAF6CC3E56C13F9E56B13F8C3E9B9
:1009FE0013F9E813F8E56B28F569E56C39F56A7AB1
:100A0E0003C3E913F9E813F8DAF7AA201A70097587
:100A1E006B00756C00020A361AEA6008EE28FEEFCB
:100A2E0039FFDAF88E6B8F6C2275E890227883E6A8
:100A3E00FFE5E820ECF7A8BDA9BE056DC3E56D94F2
:100A4E00084052756D00E9FA79A0E76044EA700734
:100A5E00E56E601B020A71C3E8956E6010E56E507C
:100A6E0006600C14020A7D0460F9020A7DE56EF53B
:100A7E006EC3946D401B755EC0C394044013755EC7
:100A8E0080C39404400B755E40C394044003755EAE
:100A9E000075BB0822E55EF46002055EE56DB407E5
:100AAE000375BB1022743279A387F0A4C5F0A2F7A8
:100ABE0033F8C3E8955E4002A85E88228824882514
:100ACE00886122753A00753B7F2275C820A8CCA993
:100ADE00CD75C824AA38AB3988388939C3E89AF855
:100AEE00E99BF9AA3AAB3BAC3AAD3B7E047F02C31D
:100AFE00EB940440021E1FC3EB940840021E1FC35A
:100B0E00ED13FDEC13FCDEF7C3EA9CFAEB9DFBEF55
:100B1E006009C3E913F9E813F8DFF7EA28FAEB39AD
:100B2E00FB8A3A8B3B400122753AFF753BFF223020
:100B3E006002613D854C50854D51D26043E6802266
:100B4E007892E6FFC3E535948240010FC3E53594F4
:100B5E00A040010FC3EF940640027F057E021E30B7
:100B6E0072010EC3E53B940350060E0E3072010E59
:100B7E00C3E53B940250060E0E3072010EA93BA83F
:100B8E003A7A04C3E913F9E813F8DAF7C3E89EF8E2
:100B9E00E99400F94009C3E89402E99400500478FE
:100BAE0002E4F9E9FBE8FAC3E913FDE813FC884C0B
:100BBE00894DC3EF94036037EF20E00DE82CF8E980
:100BCE003DF9ECFAEDFB020BEAE828F8E939F9C336
:100BDE00E89402F8E99400F97A02E4FBC3EF940377
:100BEE00400D8A4E8B4F884889498C4A8D4B2288FE
:100BFE004E894F8A488B498C4A8D4B223060028138
:100C0E000AD26043E680E52D54066027A83AA93B38
:100C1E00E53494085006E820E002A94D759100C312
:100C2E00E498F594E499F595759104D26053917F0B
:100C3E0043E68022D265753D00752000020C55D228
:100C4E0065753D00752040E52D54066002C265D2E3
:100C5E00AF206005E53D60012278017A02C3E53BD5
:0F0C6E00940540027802C3E53B940A40027803E4
:100C7D00C3E53B940F40027A03306904781E7A0174
:100C8D00206007E53D6003D2AF22D2AF0000C2AFB6
:100C9D00C3E53BFB940F40027B0FEB043073012344
:100CAD0020620123F93069027982E58BC39940D026
:100CBD00053DEAFBE59B5440B52004DBF781F020B0
:100CCD0065028155C265759100AE3AAF3BC3E49E96
:100CDD00F594E49FF595759104D26053917F43E6A9
:100CED008081553065028155D896D2AF2230690B7F
:100CFD000534206016753400020D1820600D206536
:100D0D000A206B071581158102156622A84EA94F81
:100D1D0075910053917FC3E498F594E499F5957519
:100D2D009104854850854951D26043E68022780070
:100D3D003064053065027801E53575F007A4F9E5F5
:100D4D00F028F5F0E9A2F013A2F113A2F213F53594
:100D5D00C394785003753578C3E53595364008D280
:100D6D0066D297D295D293306002A174854A508590
:100D7D004B51D26043E68022C2AFC296C294C2925A
:100D8D0030720B9002197406D5E0FD020DC3E53BE0
:100D9D0054F86022E525600A207D02C297307D025D
:100DAD00C293740FD5E0FD207D02D297307D02D223
:100DBD00937406D5E0FD207D02D296307D02D2924D
:100DCD00759F10753C02020F42C2AF207D02D29377
:100DDD00307D02D2973072179001F6C294207D02B9
:100DED00C292307D02C2967406D5E0FD020DFF90D1
:100DFD000159306206E5256002C295207D03759F7D
:100E0D0013307D03759F11753C03020F42C2AFC2B3
:100E1D0096C294C29230720B9001D37406D5E0FD48
:100E2D00020E58E53B54F86022E525600A207D024C
:100E3D00C293307D02C297740FD5E0FD207D02D2A2
:100E4D0093307D02D2977406D5E0FD207D02D292BB
:100E5D00307D02D296207D03759F11307D03759FE5
:100E6D0013753C04020F42C2AFD295307217900138
:100E7D00B0207D02C296307D02C292C2947406D516
:100E8D00E0FD020E9590014730620EE525600A20C7
:100E9D007D02C297307D02C293759F10753C05028D
:100EAD000F42C2AFC296C294C29230720B900185AE
:100EBD007406D5E0FD020EDDE53B54F86012E52524
:100ECD006002C295740FD5E0FDD2957406D5E0FD94
:100EDD00D294207D03759F13307D03759F11753C52
:100EED0006020F42C2AF207D02D297307D02D2930F
:100EFD0030721F900244207D02C296307D02C29254
:100F0D00207D02C292307D02C2967406D5E0FD02AC
:100F1D000F2290016B30620EE525600A207D02C222
:100F2D0093307D02C297207D03759F11307D03752F
:100F3D009F13753C01306B13120F5D7406D5E0FDE8
:100F4D007406D5E0FDD296D294D292C266D2AF226B
:100F5D00900145D297D295D293C296C294C292C2B5
:100F6D006222788076FF0876FF0876FF0876FF0804
:100F7D007603087604087609087601087601087666
:100F8D0001788C76010876FF0876FF0876FF0876E3
:100F9D00FF0876FF0876030876FF0876FF0876FFD0
:100FAD000876250876D00876FA0876FA08760408C9
:100FBD0076FF08760108760008767A0876FF0876BF
:100FCD0001227887E6FFC2727888E6C39403600831
:100FDD00C27DE630E102D27DC27E7889E630E10243
:100FED00D27EC3EF94026008758E01D27302100297
:100FFD00758E00C273227880E6149000809378A1DC
:10100D00F67881E6149000809378A2F6120F5D2297
:10101D007886E61490008D9378A3F6120F5D222248
:10102D00789CE67536FF75370CB402067536A075DB
:10103D00370AB4030675368275370522227896E68F
:10104D00FA7897E6FB307F047A007BFFC3EB9AFCBE
:10105D00C3948250027C82756F00056FEC856FF032
:0D106D00A4C3E5F0948040F222D27F114A26
:10107A001206DE7A007B007C101206D4E5592AFAA1
:10108A0074003BFBDCF37C04C3EB13FBEA13FADCCE
:10109A00F7FEC27F114A22E5EF20E603752000051C
:1010AA0020903FFFE520146006901DFF1460009316
:1010BA0004600375EF12C2D353D9BF7581C043FFD1
:1010CA00801206CF75EF0243B203E5B3240420E78A
:1010DA0002F5B3120F5D7580FF75A40075F1B27544
:1010EA00D4DF7590A975A5FC75F2FC75D50175A6B6
:1010FA000175E241120F6F12159878988670C2AF87
:10110A001206E81206F81206DE1206FF1206DE12B0
:10111A0007061206DE1216AC1206E81206E81206D6
:10112A00E3C2AFE4F8F6D8FD78C879C8308507D9A4
:10113A00FBD8F7021C00120F6F121598120FCF116D
:10114A0003111D112C112D1149114A78988670121C
:10115A000F5D75885075891275C82475910475D804
:10116A004075A82275B80275E690759B80759D003A
:10117A0075D10E75BC5875BB0875BA1175E8801221
:10118A0006CFD2AF12099943DA01C2D8C271120648
:10119A00E8753001D2617B037A0CE55870067A0C47
:1011AA00DB02212B1206DE207002212BC270E559C8
:1011BA00C3940240E3E52F541F855B5AF55BB55A89
:1011CA00D7DAD7C26153DACF207E0343DA20307EE2
:1011DA000343DA10C2D8C271C2757528001206E339
:1011EA00307409C3E528940A4002D2751206D478ED
:1011FA00023074027800C3E5599840F0C2AF120673
:10120A00F81206F81206F8D2AF1206E87546007808
:10121A0088E6B4030241F51206D4788CE6C3940139
:10122A0050030212F5E530C3940150030212F5206F
:10123A007435C3E55994FF50030212F5C2AF120781
:10124A000DD2AF1206E3C3E559940150EFC2AF12B3
:10125A0006F81206D91206F8D2AF1206E3C3E55908
:10126A0094FF40E90217317F05D27F114A1206E343
:10127A00C2AFC27F114AAE59C3E559947FD2AF407B
:10128A00741206CFC2AF12070DD2AFDFDC1176C3DC
:10129A00EE94057897F61206E81215DA1216B47F5C
:1012AA000AD27F114A1206E3C2AFC27F114AAE596F
:1012BA00C3E559947FD2AF50E61206CFC2AF1206E9
:1012CA00F81206D91206F8D2AFDFD61176EE240547
:1012DA007896F61206E81215DA1216E31206E311E8
:1012EA004AC3E55994FF40F4021731C3E5599546BC
:1012FA0040038559461206E378017988E7B4030268
:10130A007805C3E5599840024119C2AF12070D1278
:10131A00070D12070DD2AF1206E8753000E4F53159
:10132A00F5320531E531F470390532789AE67819E3
:10133A00146012783214600D787D14600878FA14FB
:10134A006003753200C3E53298401715327531B41F
:10135A0078998670C2AF12070DD2AF78988670124C
:10136A0006E31206D9E5297005307402212B7801AB
:10137A002074027806C3E5599840A77888E6C39492
:10138A000360031206E3E5297002212BC2AF120F94
:10139A005DE4F522F523F524F525D2AF788586623A
:1013AA00F53EF53FF540F541F542F56DF547F52C6B
:1013BA00F52DF535120AD1756D0875BB101206CFD9
:1013CA00120A37E5E820ECFBA8BDA9BEE97001F8CE
:1013DA00886E120A3B756D0875BB107887E6FE7633
:1013EA0002120FCF7887EEF6C2AF755EFF120AB30C
:1013FA0085225E85225F852260D2AF75220175241F
:10140A0001752501855D64756501D268D2697534F7
:10141A0000120EAF120EF1120AD1120AD8120B4E96
:10142A00021439120F5D120FCF756D0075BB0812C9
:10143A000C4D120CFA120D191207F7120D3B120D70
:10144A0085120AD8120B3D120B4E120C0A120C42CC
:10145A00120CFA120D191207F812095D120D3B123D
:0E146A000DD6120AD8120B3D120B4E120C0AB0
:10147800120C4D120CFA120D19120838120D3B12EB
:101488000E1A120AD8120B3D120B4E120C0A120C2D
:1014980042120CFA120D19120895120D3B120E7415
:1014A800120AD8120B3D120B4E120C0A120C4D12D6
:1014B8000CFA120D191208FA120D3B120EAF120A8D
:1014C800D8120B3D120B4E120C0A120C42120A379C
:1014D800120CFA120D19120A3B120D3B120EF112E0
:1014E8000AD8120B3D120B4E120C0A306935206BCC
:1014F8003285615E85615F855D6475650179327AE3
:101508000AC3E53499400FC269D26A8A33755EFF0F
:10151800755FFF02152BC3E5599401400302143986
:10152800021566306A1B206B18E533147004C26A12
:10153800812DF533C3E5599401400302143902158E
:1015480066C3E55C94825016307404E529600FC3C5
:10155800E53B78F0306B0278609850028139C2AF71
:10156800120F5D7887E6FE7602120FCF7887EEF6C7
:10157800E4F522F523F524F525F562C268D2AF1209
:1015880006CF120F5D307406E5297002212B612702
:10159800901A0D782012161CE520B45A0CA31216C6
:1015A8001CE520B4A5030215BA120F6F1215DA0252
:1015B80015D9901A0378807B0A12161CA308DBF948
:1015C800901A0F788C7B1512161CA308DBF9901A59
:1015D8002422C2AF12165B121635901A00740D122F
:1015E8001621A37402121621A37413121621901A3D
:1015F8000378807B0A121620A308DBF9901A0F786B
:101608008C7B15121620A308DBF912166E12164CE5
:10161800901A2422E493F622E6438F01538FFD7536
:10162800EF0275B7A575B7F1F0538FFE22438F020D
:10163800438F0175EF0275B7A575B7F1901A0DF0D4
:10164800538FFC22901A0D745AD121901A0E74A54A
:10165800D121227A3079D07820901A40D11CE52007
:10166800F709A3DAF7227A3079D0901A40E7D12126
:1016780009A3DAF922AB71A872BB01027984BB0213
:10168800027985BB03027986BB04027992BB050205
:101698007987BB0602799CBB07027988BB08027967
:1016A80089E8F7227C051206E8DCFB22C2AF1206A5
:1016B800F81206FF12070612070D1206D91206F8CD
:1016C8001206FF12070612070D1206D91206F812A3
:1016D80006FF12070612070DD2AF22C2AF12070D7E
:1016E8001207061206FF1206F81206D912070D1283
:1016F80007061206FF1206F81206D912070D12077E
:10170800061206FF1206F8D2AF22AE71AF72C2AF50
:101718001206F81206F81206F81206D9DEF21207B7
:101728000D1206D9DFF8D2AF22D1B4D1ACD1AC7545
:101738007101757201757300F1127C05AD591206BD
:10174800E8C3ED955970F5C3E5599401400AC3E51E
:101758005994FF403202176DD17DB1DAD1B4C2AFCE
:1017680075EF12D1ACDCD50573C3E5739403500251
:1017780080C6D1AC0572E5711490009A93F808C33D
:10178800E57298500280AED1ACD1AC0571C3E57159
:1017980094095002809C120F6FB1DAC2AF75EF1234
:0217A800D1ACC2
:101A00000D0213FFFFFFFF0304090101015AA501A5
:101A1000FFFFFFFFFF03FFFFFF25D0FAFA04FF01DE
:051A2000007AFF01FF48
:101A400023536B79494949333041232020202020FA
:101A500023424C48454C4923463333302320202031
:101A60002020202020202020202020202020202076
:101C0000C2AFC2D353D9BF7581C043B20343FF8073
:101C1000752438752503B1BF75EF0275E24043F1B5
:101C20002053A4DFD285780379E67C1075220075F5
:101C30002300901DCC7B0675249875250130850204
:101C4000813D208508D8FBD9F9DCF781AD308508C6
:101C5000D8FBD9F9DCF781ADB17FE493A3C39A60D7
:101C6000028126DBDDB171600281267B08E493FAF4
:101C7000A3B152DBF87A30B152752200752300B15E
:101C800071EAFCEBFDC3ED94FE400EB1718A278B27
:101C900028ED30E0048A828B83B1717AC270D8C398
:101CA000ED94FE601050CEBD0022EC600675200061
:101CB0000200008100A827A9280809D804D90281B8
:101CC000C9B175EA89AAF281BB0D8199C3ED94036C
:101CD0005049EDA2E092007AC5C3E5829400E58305
:101CE000941C5093200010438F02438F0175B7A5B9
:101CF00075B7F1F030001FA827A9280809438F0104
:101D0000538FFDD804D902A11689AAE275B7A5752B
:101D1000B7F1F0A3A103538FFC81757AC1BD030C09
:101D2000E493A3FAB136DCF8B12E81758177AA224B
:101D3000AB23B152EBFAEA6222752608C3E52313FE
:101D4000F523E52213F52250066323A0632201D573
:101D500026EAB1BFB1BF75260AEAF4200102D28596
:101D6000300102C285B1BFC3134002C201D526EBC8
:101D700022B175EAFB208502A175308502A17A7532
:101D80002608AE24AF25C3EF13FFEE13FEB1C3B197
:101D9000BFC3EA133085024480FA30E703632201AF
:101DA000C3E52313F523E52213F52250066323A090
:101DB000632201D526D9E52265236523F52222AECB
:101DC00024AF250E0FDEFEDFFCD20122424C486517
:0A1DD0006C6934373132F33006013C
:00000001FF
